:02000000CA280C
:10000800DF00030E8301C2000A08C1008A010B1D2C
:100018001E2883120430850605191A280130A70006
:100028003B08BC003B08FF3C81001D283C08053EFE
:1000380081000B1183120C1C2928F8308F003030F6
:100048008E000C10BE0A0319BF0A41088A00420E2E
:080058008300DF0E5F0E0900BA
:0C00600007308312DD00DD0B33280800A0
:10006C0082308312DC00DD30DD00DD0B3B28DC0B45
:08007C003B2800000000080011
:10008400C33083129F05F0309F05BF309F05F030C9
:1000940083169F0483129F174508D000D00D50107B
:1000A400D00D501050089F041F1430209F149F1C23
:1000B4005D28000059281F101E08D100D0018316A6
:1000C4001E085004C6005108C7000030C704460883
:0800D400D0004708D10008002C
:1000DC00831203132230DC00D801D901DA01DB01D1
:1000EC00DC030319A4280310DB0CDA0CD90CD80C94
:1000FC00D30CD20CD10CD00C031C7628DC030319C6
:10010C0096285408D80755080318550FD9075608D0
:10011C000318560FDA0757080318570FDB077A280E
:10012C005408D80755080318550FD9075608031853
:0E013C00560FDA0757080318570FDB070800A5
:10014A0083169C1CAA280000A52845089B0046087F
:10015A009A009C131C150B08D0008B1355309D0078
:10016A00AA309D009C14D01BBC288B13BD288B176A
:04017A001C1108004C
:10017E008312450883169B009C131C141A08D10089
:06018E005108D00008003A
:10019400073083129900393083169F0005148514A3
:1001A40005110516851283121F179F159F178512B7
:1001B40005156430C000BC01BB01BE01BF015F3046
:1001C400831681008B16BD01362036206400851904
:1001D400072936203620C50142205008C3005108A3
:1001E400C400C5014308C600A52036208516043086
:1001F400DB008E30DC001230DD00DD0BFF28DC0B71
:10020400FF28DB0BFF280000851264003620C5019F
:10021400BF205008BD0050081F3C03181229BD011F
:10022400831290121012901030308E00F8308F002C
:100234000C10AC01AD01C301C401B101B201B301A1
:10024400B40183160C140B178B17831210140A3085
:10025400BB00FF30B000AE01AF01AA01AB01A401A5
:10026400A501A201A30164000230DB008630DC009A
:100274009930DD00DD0B3C29DC0B3C29DB0B3C29F0
:1002840085160230DB008630DC009930DD00DD0BA2
:100294004929DC0B4929DB0B4929851264003E08F6
:1002A400A0003F08A10024083E02D1002508031C39
:1002B400013E3F02D2005208003C031D632951084D
:1002C400400203186C2983122008A4002108A50009
:1002D400203085062E08A8002F08A9002C08AE009F
:1002E4002D08AF00A7012708003A03197529C50195
:1002F40042205008C3005108C4000330C500422006
:100304005008AC005108AD00A601C50142205008B8
:10031400B9005108BA000330C50042205008A000BB
:100324005108A1005008AC0751080318013EAD075D
:10033400AD0CAC0CAD133A084402031DA3293908D3
:1003440043020318A9293908C3003A08C40026083F
:10035400033A0319AF29A60A8729AC0DAD0D2C1059
:10036400AC0DAD0D2C103E08A0003F08A1002A08DA
:100374003E02D1002B08031C013E3F02D200003094
:100384005202031DC7290F3051020318CA29422AF9
:1003940064002008AA002108AB003108B500320827
:1003A400B6003308B7003408B8002C08D0002D0874
:1003B400D100D201D3014308D4004408D500D601AA
:1003C400D7016E205008B1005108B2005208B300A2
:1003D4005308B4004408003C031DF22943083D02BD
:1003E40003181E2A34083806031D022A3308370668
:1003F400031D022A32083606031D022A3108350677
:10040400031D072AFA30C000422A38083402031DAB
:10041400152A37083302031D152A36083202031D34
:10042400152A3508310203181B2A9630C000B0097A
:100434001D2A9630C0002B2A6430C0000A30BB004D
:10044400FF30B000B101B201B301B401C301C40172
:10045400422A30080319382AFA303B020318342A96
:10046400BB0A372AFA30BB00B001422A3B080A3CD7
:1004740003183E2ABB03422A0A30BB00FF30B000F7
:040484005129432A8D
:02400E00DC31A3
:020000040000FA
:104200000400FF00FF000000FF00FF00FF00FF00B0
:10421000FF00FF00FF00FF00FF00FF00FF00FF00A6
:10422000FF00FF00FF00FF00FF00FF00FF00FF0096
:10423000FF00FF00FF00FF00FF00FF00FF00FF0086
:10424000FF00FF00FF00FF00FF00FF00FF00FF0076
:10425000FF00FF00FF00FF00FF00FF00FF00FF0066
:10426000FF00FF00FF00FF00FF00FF00FF00FF0056
:10427000FF00FF00FF00FF00FF00FF00FF00FF0046
:10428000FF00FF00FF00FF00FF00FF00FF00FF0036
:10429000FF00FF00FF00FF00FF00FF00FF00FF0026
:1042A000FF00FF00FF00FF00FF00FF00FF00FF0016
:1042B000FF00FF00FF00FF00FF00FF00FF00FF0006
:1042C000FF00FF00FF00FF00FF00FF00FF00FF00F6
:1042D000FF00FF00FF00FF00FF00FF00FF00FF00E6
:1042E000FF00FF00FF00FF00FF00FF00FF00FF00D6
:1042F000FF00FF00FF00FF00FF00FF00FF00FF00C6
:00000001FF
